:100000000C94280018950000189500001895000021
:10001000189500001895000018950000189500002C
:10002000189500000C94700C1895000018950000AD
:10003000189500001895000018950000189500000C
:1000400018950000189500001895000018950000FC
:100050008FE181BD87E181BD8FE58DBFC4E0E8E719
:100060004E2E88E08EBFD8E0F7E05F2EEEEFF7E08F
:10007000A0E6B0E088278D933197E9F783E389B94B
:1000800088E18AB9662481E48ABB81E38BBB8FEB6C
:1000900087BB8FEB88BB88E084BB83E085BB80E0B7
:1000A00081BB8BE382BB80E08FBD81E08EBD8FE1A1
:1000B00081BD87E181BD86E086B980E487B9C398B8
:1000C000C29AD89ADE9AC498C798C598F894A89509
:1000D0007091CF0078607093CF007091CF007B7FDC
:1000E0007093CF000027AFECB0E08C9183FB0EF44F
:1000F00001E041E0041781E009F080E08F930027E0
:10010000AFECB0E08C9182FB0EF401E041E004170B
:1001100081E009F080E09F91892B882311F40C94F1
:100120009400DC9881E58ABB0E949F0D7091CF00FE
:1001300070627093CF00EFEFF1E0A0ECB0E091E0DF
:100140000E94EC2D0091C000003081E009F080E0B9
:100150008F930091C0000E3F80E010F009F081E025
:100160009F91892B882311F40C94B9008EEB809316
:10017000C0000091C0004AE0040F01BF89E190E097
:100180000E94DE2CDC9AEEE2FCE50E94252C002782
:10019000AFECB0E08C9183FB0EF401E041E004177A
:1001A00011F00C94DB00EAE4FCE50E94252C0E948F
:1001B000312C0C94EE00ECE4FCE50E94252CAFEC15
:1001C000B0E08C9182FBA8E6B7E00E94032D8D93EE
:1001D00088278C930E941D2C0E94312CEAE0F0E0CD
:1001E000BB27A0E10E94E92D073411F40C942E01E5
:1001F000EBE0F0E0A0E1BB278FE08C937BE70E946F
:10020000D82DECE0F0E001E010E0A0E1BB277BE7B7
:100210000E94DA2DEAE0F0E0A0E1BB2787E48C93AE
:100220007BE70E94D82DEEE0F0E0A0E1BB2780E064
:100230008C937BE70E94D82DE0E1F0E000E010E035
:10024000A0E1BB277BE70E94DA2DEFE0F0E0A0E120
:10025000BB2780E08C937BE70E94D82DEBE0F0E099
:10026000ABEBB0E00E94E92D0091BB00043618F022
:1002700011F00C943D010C94400184E68093BB0086
:1002800080E797E9ACEBB0E08D939C93ECE0F0E075
:10029000A6EBB0E00E94EB2DEEE0F0E0A1ECB0E0C8
:1002A0000E94E92DEFE0F0E0A2ECB0E00E94E92D21
:1002B0000E94A30DE0E1F0E0A3E6B0E00E94EB2D88
:1002C000A3E6B0E00E948C2BE0E1F0E0A3E6B0E012
:1002D0007BE70E94DA2DA6EBB0E00D911C91003077
:1002E00050E0150711F00C947B0181E090E0A6EB43
:1002F000B0E08D939C93EEE4FCE50E94252CA8E6EB
:10030000B7E0EBEBF0E00E94712D0E941D2CE6E5BA
:10031000FCE50E94252CA8E6B7E0E6EBF0E00E94A1
:10032000622D0E941D2CE6E5FCE50E94252CA8E626
:10033000B7E0E1ECF0E00E94712D0E941D2CE6E593
:10034000FCE50E94252CA8E6B7E0E2ECF0E00E9474
:10035000712D0E941D2CE6E5FCE50E94252CA8E6E7
:10036000B7E0E3E6F0E00E94622D0E941D2C0E949F
:10037000312C80E08093CE0070916A00777F70937B
:100380006A0080E08093C40086E08093BE008DE028
:100390008093BF00E9E6F0E0FA93EA930E94C11C63
:1003A000229684E190E00E94DE2CDE980E94CA2C06
:1003B000C49AE8E5FCE50E94252C0E94312C88ECCB
:1003C00090E00E94DE2CA89581B5886181BD877F71
:1003D00081BDE0E6F0E0FA93EA930E9409212296BB
:1003E000A89500916000003011F40C9403020E9463
:1003F0004B20E2E6FCE50E94252C0E94312C0E9455
:10040000660D0C9408027091CF007F7B7093CF0033
:10041000ECE6FCE50E94252C0E94742084E690E026
:100420000E94DE2C00916900003018F011F00C944D
:100430001B020C942202E9E6F0E0FA93EA930E9490
:10044000501E22960027AFECB0E08C9186FB0EF494
:1004500001E040E0041711F00C9430020E94FE13FA
:100460008FEF0E94342CDC9882E390E00E94DE2C17
:100470007894A89581B5886081BDA2EBB0E04D91DC
:100480005C91A6EBB0E00D911C910417150718F0D4
:1004900011F00C944D020C94530281E090E0A6EB15
:1004A000B0E08D939C930027AAE6B0E08C9184FB8A
:1004B0000EF401E041E0041781E009F080E08F9341
:1004C0000027AFECB0E08C9186FB0EF401E040E039
:1004D000041781E009F080E09F918923882311F4BB
:1004E0000C948502E6EBF0E0FA93EA935A924A9272
:1004F00080E0A42DB52D8C9381E00E94792B0E9481
:10050000E011249681E00E94752B80E08093B80072
:1005100080E08093690070916A007F7770936A0031
:100520000027AFECB0E08C9186FB0EF401E041E0D7
:10053000041711F00C949E020E949F0DA895ABE643
:10054000B0E088278C930027AFECB0E08C9183FB60
:100550000EF401E041E0041711F00C94B6020E9481
:10056000152CABE6B0E08D9388278C93ABE6B0E01A
:100570008C91803011F00C9461050091CE00003018
:1005800081E009F080E08F930027AAE6B0E08C912B
:1005900081FB0EF401E040E0041781E009F080E007
:1005A0009F91892B882311F40C944504E0E6F0E038
:1005B000FA93EA930E94191D229600916000003080
:1005C00018F011F00C94E6020C94450470916A0046
:1005D000706870936A000091D000003011F00C94A4
:1005E00042034091C40000916000041718F011F01C
:1005F0000C94FC020C944203809160008093C40030
:100600000027AAE6B0E08C9184FB0EF401E040E004
:10061000041711F00C941C03A0E6B0E08C91A6EB3B
:10062000B0E08D9388278C93ABE6B0E0E6E7FCE57D
:100630000E94042C0C9442030027AFECB0E08C9194
:1006400087FB0EF401E041E0041711F00C943C0329
:10065000A0E6B0E00D91112741E050E0040F151F16
:10066000A6EBB0E00D931C93ABE6B0E0E6E7FCE54B
:100670000E94042C0C944203ABE6B0E0E8E7FCE5F2
:100680000E94042C0091D000013011F00C94C203A0
:1006900000916000013011F00C945403ABE6B0E01F
:1006A000E8E7FCE50E94042C00916000023011F0A4
:1006B0000C946003ABE6B0E0EAE7FCE50E94042C92
:1006C00080E08093620000916000033081E009F0D7
:1006D00080E08F930091BB00043681E008F080E059
:1006E0009F918923882311F40C947E03ABEBB0E037
:1006F0008C918E5F8C9381E080936200009160000A
:10070000043081E009F080E08F930091BB0002305B
:1007100080E010F009F081E09F918923882311F493
:100720000C949A03ABEBB0E08C9182508C9381E0F7
:100730008093620000916200013011F00C94C203BA
:100740008EB5887F8EBD5A924A928091BB00A42DAF
:10075000B52D8C9381E00E94792B0E94F727229679
:1007600081E00E94752BEBE0F0E0ABEBB0E07BE7C3
:100770000E94D82D0091CE00013011F00C94C203DC
:1007800081E08EBD0091D000023011F00C94450440
:100790004091C40000916000041718F011F00C940F
:1007A000D3030C944504809160008093C4000091B1
:1007B0006000013011F00C94E90381E090E0A6EBB9
:1007C000B0E08D939C93ABE6B0E0E6E7FCE50E94D9
:1007D000042C00916000023011F00C942D04A2EB67
:1007E000B0E00D911C9141E050E0041B150BA3E615
:1007F000B0E00D931C9302E010E00F931F93A3E66B
:10080000B0E08D919C918A939A930E94A52B229699
:10081000402F512F1F910F91040F151FA3E6B0E039
:100820000D931C93A6EBB0E04D915C91A3E6B0E074
:100830000D911C910417150711F40C94EF03A3E616
:10084000B0E08D919C91A6EBB0E08D939C93ABE6CC
:10085000B0E0E6E7FCE50E94042C00916000033064
:1008600011F00C943904ABE6B0E0E8E7FCE50E9437
:10087000042C00916000043011F00C944504ABE6A8
:10088000B0E0EAE7FCE50E94042C0027AAE6B0E00D
:100890008C9184FB0EF401E041E0041781E009F043
:1008A00080E08F930027AFECB0E08C9187FB0EF4D3
:1008B00001E041E0041781E009F080E09F91892385
:1008C0008F930091CE00013081E009F080E09F918C
:1008D0008923882311F40C94B004A6EBB0E00D91A9
:1008E0001C91013050E0150711F00C94B004E0E6C3
:1008F000F0E0FA93EA930E94191D2296009160009D
:10090000003080E010F009F081E08F93A2EBB0E0BE
:100910004D915C91A0E6B0E00D91112704171507E9
:1009200081E008F080E09F918923882311F40C94E2
:10093000B004A0E6B0E00D91112741E050E0040FB3
:10094000151FA6EBB0E00D931C93ABE6B0E0E6E715
:10095000FCE50E94042C70916A00706870936A0034
:100960000027AAE6B0E08C9180FB0EF401E040E0A5
:10097000041711F00C946105E9E6F0E0FA93EA93AC
:100980000E94C11C229600916900043011F00C9461
:10099000D0040E94570D70916A00706870936A00CD
:1009A00080E08093600000916900023081E009F0EE
:1009B00080E08F930091BB00043681E008F080E076
:1009C0009F918923882311F40C94EE04ABEBB0E0E3
:1009D0008C918B5F8C9381E0809360000091690023
:1009E000033081E009F080E08F930091BB00053077
:1009F00081E009F080E09F918923882311F40C9411
:100A0000070581E08093BB0081E080936000009146
:100A10006900033081E009F080E08F930091BB0012
:100A2000053080E010F009F081E09F918923882350
:100A300011F40C942305ABEBB0E08C9185508C93B2
:100A400081E08093600000916000013011F00C940F
:100A500050058EB5887F8EBD5A924A928091BB0018
:100A6000A42DB52D8C9381E00E94792B0E94F7274D
:100A7000229681E00E94752BEBE0F0E0ABEBB0E05A
:100A80007BE70E94D82D0091CE00013011F00C942C
:100A90004B0581E08EBD70916A00706870936A00AA
:100AA00000916900013011F00C946105ABE6B0E0F3
:100AB000E8E7FCE50E94042C70916A00706870936E
:100AC0006A00EBE6F0E0ABE6B0E00E94F72CABE6A4
:100AD000B0E08C91803081E009F480E08F93009148
:100AE0006900003081E009F480E09F91892B8F93A9
:100AF0000091B800013081E009F080E09F91892BDE
:100B0000882311F40C9490020091B800013011F088
:100B10000C94AB0580E08093B800ABE6B0E0E8E76A
:100B2000FCE50E94042C0027AFECB0E08C9187FB21
:100B30000EF401E041E0041711F00C94AB0581E0E4
:100B400090E0A6EBB0E08D939C93ABE6B0E0E6E7D7
:100B5000FCE50E94042CABE6B0E0ECE7FCE50E946B
:100B6000032E11F00C94F2055A924A928091BE0025
:100B7000A42DB52D8C9381E00E94792B5A924A9234
:100B80008091BF00A42DB52D8C9381E00E94792B1C
:100B90000E945028249682E00E94752B0091C2008A
:100BA00041E0042BA0E6B0E00C937091CF0070619F
:100BB0007093CF008EB5887F8EBDEFE0F0E0A0E6A9
:100BC000B0E07BE70E94D82D809160008093C20046
:100BD0000091CE00013011F00C94F00581E08EBD43
:100BE0000C94A20BEEE7FCE50E94032E11F00C948E
:100BF00035065A924A9280E0A42DB52D8C9381E05F
:100C00000E94792B5A924A9280E0A42DB52D8C93A4
:100C100081E00E94792B0E945028249682E00E9455
:100C2000752B0091C2004EEF0423A0E6B0E00C93B8
:100C30007091CF007F7E7093CF008EB5887F8EBD80
:100C4000EFE0F0E0A0E6B0E07BE70E94D82D8091D5
:100C500060008093C2000091CE00013011F00C942E
:100C6000330681E08EBD0C94A20BE6E7FCE50E9402
:100C7000032E11F00C94A5060091CE00013011F066
:100C80000C9444060E94570DA2EBB0E04D915C918C
:100C9000A6EBB0E00D911C910417150718F011F0A8
:100CA0000C94A0060027AFECB0E08C9186FB0EF40C
:100CB00001E040E0041711F00C947106E6EBF0E05F
:100CC000FA93EA935A924A9280E0A42DB52D8C9320
:100CD00081E00E94792B0E94E011249681E00E941D
:100CE000752B0027AFECB0E08C9186FB0EF401E091
:100CF00041E0041711F00C949E060E94660D002737
:100D0000AFECB0E08C9186FB0EF401E040E00417FC
:100D100011F00C949E06E6EBF0E0FA93EA935A92F7
:100D20004A9280E0A42DB52D8C9381E00E94792B0E
:100D30000E94E011249681E00E94752B0C94A3067A
:100D400080E08093C4000C94A20BE0E8FCE50E94D4
:100D5000032E11F00C94B3060E94570D80E080938F
:100D6000C4000C94A20BE2E8FCE50E94032E11F0F3
:100D70000C94ED060091CE00013011F00C94EB06BE
:100D80000027AAE6B0E08C9183FB0EF401E040E07E
:100D9000041711F00C94DD068EB5887F8EBD89B7DF
:100DA0008B7F89BF70916A00786070936A0084E6D7
:100DB00090E00E94DE2C0C94EB0670916A00777F25
:100DC00070936A0080E29EE49DBD8CBD81E08EBD83
:100DD00089B7846089BF0C94A20BE8E7FCE50E9408
:100DE000032E11F00C9485070091CE00013011F014
:100DF0000C94FC060E94570DA6EBB0E00E948C2BD1
:100E00000027AFECB0E08C9185FB0EF401E041E0EF
:100E1000041711F00C9421070027AAE6B0E08C918A
:100E200084FB0EF401E040E0041711F00C941C0761
:100E3000A6EBB0E00E94922B7091CF007F7D709363
:100E4000CF00A2EBB0E04D915C91A6EBB0E00D912C
:100E50001C910417150718F011F00C9431070C942D
:100E6000370781E090E0A6EBB0E08D939C930027DC
:100E7000AFECB0E08C9186FB0EF401E040E004178B
:100E800011F00C945607E6EBF0E0FA93EA935A92CD
:100E90004A9280E0A42DB52D8C9381E00E94792B9D
:100EA0000E94E011249681E00E94752B0027AFEC90
:100EB000B0E08C9186FB0EF401E041E0041711F0E4
:100EC0000C9483070E94660D0027AFECB0E08C9174
:100ED00086FB0EF401E040E0041711F00C94830748
:100EE000E6EBF0E0FA93EA935A924A9280E0A42D5E
:100EF000B52D8C9381E00E94792B0E94E0112496FD
:100F000081E00E94752B0C94A20BEAE7FCE50E949D
:100F1000032E11F00C94FD070091CE00013011F06A
:100F20000C9494070E94570DA6EBB0E00D911C9114
:100F3000013050E0150718F011F00C94A1070C9443
:100F4000A707A6EBB0E00E94922B0C94AF07A2EB90
:100F5000B0E08D919C91A6EBB0E08D939C9300271F
:100F6000AFECB0E08C9186FB0EF401E040E004179A
:100F700011F00C94CE07E6EBF0E0FA93EA935A9264
:100F80004A9280E0A42DB52D8C9381E00E94792BAC
:100F90000E94E011249681E00E94752B0027AFEC9F
:100FA000B0E08C9186FB0EF401E041E0041711F0F3
:100FB0000C94FB070E94660D0027AFECB0E08C910B
:100FC00086FB0EF401E040E0041711F00C94FB07DF
:100FD000E6EBF0E0FA93EA935A924A9280E0A42D6D
:100FE000B52D8C9381E00E94792B0E94E01124960C
:100FF00081E00E94752B0C94A20BE4E8FCE50E94B2
:10100000032E11F00C947008A6EBB0E00E948C2B1C
:10101000A2EBB0E04D915C91A6EBB0E00D911C917C
:101020000417150718F011F00C9418080C941E08FA
:1010300081E090E0A6EBB0E08D939C938EB5887F25
:101040008EBDA2E7B0E00D911D912D913C91A2E9DA
:10105000B0E00D931D932D933C930027AFECB0E0CF
:101060008C9186FB0EF401E040E0041711F00C9423
:1010700066085A924A92A2E9B0E00D911D912D9115
:101080003C91A42DB52D0D931D932D933C9384E09D
:101090000E94792B5A924A92A6EBB0E08D919C91D6
:1010A000A42DB52D8D939C9382E00E94792B5A92AA
:1010B0004A9280E0A42DB52D8C9381E00E94792B7B
:1010C0000E940D15269687E00E94752B0091CE0098
:1010D000013011F00C946E0881E08EBD0C94A20BCF
:1010E000ECE4FCE50E94032E11F00C94E408A6EB5E
:1010F000B0E00D911C91013050E0150718F011F08F
:101100000C9484080C948A08A6EBB0E00E94922B01
:101110000C949208A2EBB0E08D919C91A6EBB0E00C
:101120008D939C938EB5887F8EBDA2E7B0E00D9124
:101130001D912D913C91A2E9B0E00D931D932D934B
:101140003C930027AFECB0E08C9186FB0EF401E0FD
:1011500040E0041711F00C94DA085A924A92A2E97E
:10116000B0E00D911D912D913C91A42DB52D0D93C5
:101170001D932D933C9384E00E94792B5A924A92BE
:10118000A6EBB0E08D919C91A42DB52D8D939C93F1
:1011900082E00E94792B5A924A9280E0A42DB52DCC
:1011A0008C9381E00E94792B0E940D15269687E092
:1011B0000E94752B0091CE00013011F00C94E208D2
:1011C00081E08EBD0C94A20BE6E8FCE50E94032EA4
:1011D00011F00C94F408ECE0F0E0A6EBB0E07BE753
:1011E0000E94DA2D0C94A20BE8E8FCE50E94032E85
:1011F00011F00C9408098DE181BD85E181BD0E944B
:10120000570D81B5886081BD0C9404090C94A20B24
:10121000ABE6B0E0EAE8FCE50E94032E81E008F4CA
:1012200080E08F93ABE6B0E0ECE8FCE50E94032E93
:1012300081E010F009F080E09F918923882311F468
:101240000C94DC0989B78B7F89BF8EB5887F8EBDF2
:101250000E94112CA0E6B0E08C9300916000003059
:1012600011F40C9428090E94152CA6EBB0E08D9384
:1012700088278C9380E08093CE0070916A00777FFE
:1012800070936A00A2EBB0E04D915C91A6EBB0E0E8
:101290000D911C910417150780E010F009F081E012
:1012A0008F93A6EBB0E00D911C91003050E0150734
:1012B00081E009F080E09F91892B882311F40C9440
:1012C0007C0981E090E0A6EBB0E08D939C93E6EB87
:1012D000F0E0FA93EA935A924A9281E0A42DB52D58
:1012E0008C9381E00E94792B0E94E011249681E08A
:1012F0000E94752B0C94DA090027AFECB0E08C91BA
:1013000086FB0EF401E040E0041781E009F080E084
:101310008F93ABE6B0E0EAE8FCE50E94032E81E0A3
:1013200009F080E09F918923882311F40C94AB0984
:10133000E6EBF0E0FA93EA935A924A9281E0A42D08
:10134000B52D8C9381E00E94792B0E94E0112496A8
:1013500081E00E94752B0027AFECB0E08C9186FBFA
:101360000EF401E040E0041781E009F080E08F9383
:10137000ABE6B0E0ECE8FCE50E94032E81E009F06A
:1013800080E09F918923882311F40C94DA09E6EB1D
:10139000F0E0FA93EA935A924A9280E0A42DB52D98
:1013A0008C9381E00E94792B0E94E011249681E0C9
:1013B0000E94752B0C94A20BEEE8FCE50E94032E14
:1013C00011F00C94170A0E94112CA0E6B0E08C9347
:1013D00000916000003011F40C94E3090E94152C78
:1013E000ABEBB0E08C938EB5887F8EBD5A924A925B
:1013F0008091BB00A42DB52D8C9381E00E94792BA8
:101400000E94F727229681E00E94752BEBE0F0E026
:10141000ABEBB0E07BE70E94D82D0091CE0001300D
:1014200011F00C94150A81E08EBD0C94A20BE0E93A
:10143000FCE50E94032E11F00C94650A0E94112C09
:10144000A0E6B0E08C9300916000003011F40C94A1
:101450001E0A8091C100809360000E94152CA1ECAF
:10146000B0E08C93A1ECB0E08C918F738C930E94D0
:10147000A30D0091C10040E10423A0E6B0E00C936D
:1014800000916000003111F00C944A0A0E949F0DF7
:101490000C944C0A0E94A10DA1ECB0E08C918F7EBF
:1014A0008C938EB5887F8EBDEEE0F0E0A1ECB0E0CD
:1014B0007BE70E94D82D0091CE00013011F00C94F2
:1014C000630A81E08EBD0C94A20BEAE4FCE50E9465
:1014D000032E11F00C94D30A0091C1004FE30423B2
:1014E000A0E6B0E00C930091CE00013011F00C9416
:1014F0007E0AA0E6B0E08C9180588C930027AFEC78
:10150000B0E08C9186FB0EF401E041E0041711F08D
:101510000C948F0AA0E6B0E08C91805C8C9300273D
:10152000AAE6B0E08C9183FB0EF401E041E00417E1
:1015300011F00C94A00AA0E6B0E08C91805E8C9330
:101540008091B600809362008EB5887F8EBDDC9A54
:1015500082E090E00E94DE2C31E0A0E6B0E00E9444
:101560002C2C31E0ABEBB0E00E942C2C31E0A2E659
:10157000B0E00E942C2C8091B2008093620031E098
:10158000A2E6B0E00E942C2C83E090E00E94DE2CCA
:10159000DC980091CE00013011F00C94D10A81E06A
:1015A0008EBD0C94A20BE2E9FCE50E94032E11F023
:1015B0000C94600BA5EDB0E00D911D912D913C9127
:1015C000A1EDB0E04D915D916D917C910E944A2D0D
:1015D000A5E6B0E00D931D932D933D93A5E6B0E0F5
:1015E0000E947D2BA5E6B0E00D911D912D913C91BF
:1015F00040E052E060E070E00E943E2CA5E6B0E0E2
:101600000D931D932D933D93A5E6B0E00D911D9193
:101610002D913C91A3ECB0E04C915527662777279C
:101620000E94432CA5E6B0E04D935D936D937D93AE
:10163000A5E6B0E00D911D912D913C914AE050E05E
:1016400060E070E00E94432CA5E6B0E04D935D930E
:101650006D937D9344E150E060E070E0A5E6B0E07A
:101660000D911D912D913C910E944F2D0CF402C0C3
:101670000C94440B00E010E020E030E0A5E6B0E080
:101680000D931D932D933C938EB5887F8EBDDC9A70
:1016900082E090E00E94DE2C34E0A5E6B0E00E94FB
:1016A0002C2C83E090E00E94DE2CDC980091CE0090
:1016B000013011F00C945E0B81E08EBD0C94A20BF6
:1016C000E4E9FCE50E94032E11F00C94820B8EB528
:1016D000887F8EBDDC9A82E090E00E94DE2CA4EA36
:1016E000B0E00E941F2C83E090E00E94DE2CDC988A
:1016F0000091CE00013011F00C94800B81E08EBD82
:101700000C94A20BE6E9FCE50E94032E11F00C9468
:10171000A20B8EB5887F8EBDDC9A82E090E00E949D
:10172000DE2C0E94A91483E090E00E94DE2CDC985D
:101730000091CE00013011F00C94A00B81E08EBD21
:101740000C94A20B81E090E00E94DE2C0027AAE618
:10175000B0E08C9187FB0EF401E040E0041718F034
:1017600011F00C94B50B0C946E0C009169000030D4
:1017700018F011F00C94BE0B0C94250CA895E0E623
:10178000F0E0FA93EA930E94C11C22960091600057
:10179000043011F00C94190C0E94570D80E08093D6
:1017A000C4000E94A10D85E090E00E94DE2C80E044
:1017B00080936200E0E6F0E0FA93EA930E94C11C95
:1017C0002296A2E6B0E08C918F5F8C9388E090E047
:1017D0000E94DE2C00916000003081E009F080E082
:1017E0008F9300916200043680E010F009F081E0F0
:1017F0009F91892B882311F40C94DA0B00916200DD
:10180000043618F011F00C94070C0C94160C81B5EA
:10181000886181BD877F81BDE3E6F0E0FA93EA93BA
:101820000E94580E229681B5886081BD80E0809329
:10183000600081E090E00E94DE2C009160000030AA
:1018400011F00C94BE0B0C94640C0091D00001308C
:1018500011F00C94600C80E090E0A3E6B0E08D9372
:101860009C93E0E6F0E0FA93EA930E94191D229619
:10187000A3E6B0E00E948C2BEF93FF93ECE8F1E03D
:101880000E94B22CFF91EF9100916000003081E046
:1018900009F080E08F93A3E6B0E00D911C9108322F
:1018A00050E0150780E010F009F081E09F91892B4E
:1018B000882311F40C94310C81E090E00E94DE2C1E
:1018C00081E090E00E94DE2C0091CE00003011F00B
:1018D0000C946E0C85E090E00E94DE2C0C948B0240
:1018E0000F921F922F923F924F925F927F928F9210
:1018F0009F92AF92BF920F931F932F933F934F935B
:101900005F936F937F938F939F93AF93BF93CF9387
:10191000DF93EF93FF938FB78F93F89489B78B7F03
:1019200089BF8EB5887F8EBD5A924A9280E092E040
:10193000A42DB52D8D939C9382E00E94792B0E945B
:10194000F32A229682E00E94752B0091D9000A307A
:1019500011F00C94AD0C0E949F0D0E943D2400914B
:10196000D9000A3011F00C94BA0C0E94A10D80E04D
:101970008093D900A9EDB0E08C918F5F8C93A895EE
:101980000027AFECB0E08C9186FB0EF401E040E064
:10199000041711F00C94DF0C5A924A9280E092E006
:1019A000A42DB52D8D939C9382E00E94792B0E94EB
:1019B000F32A229682E00E94752B0E943D24A5ED19
:1019C000B0E04D915D916D917C91A1EDB0E00D91F4
:1019D0001D912D913C910E944F2D80E00CF481E0EF
:1019E0008F930027AFECB0E08C9186FB0EF401E002
:1019F00040E0041781E009F080E09F91892388236B
:101A000011F40C940E0D80E49CE99DBD8CBD81E029
:101A10008EBD89B7846089BF0C94370D80E08093B8
:101A2000CE0070916A00777F70936A000027AFEC58
:101A3000B0E08C9186FB0EF401E040E0041711F059
:101A40000C942B0DAAE6B0E08C9184FBA8EBB0E0DF
:101A5000882780F98C930091C1004FE70423A1E609
:101A6000B0E00C930E94A10D80E08093C4008F91A0
:101A70008FBFFF91EF91DF91CF91BF91AF919F9178
:101A80008F917F916F915F914F913F912F911F9116
:101A90000F91BF90AF909F908F907F905F904F90ED
:101AA0003F902F901F900F901895F894FFCF89B713
:101AB0008B7F89BF8EB5887F8EBD80E08093CE00FE
:101AC00070916A00777F70936A000895DE9A6E982D
:101AD000C498C598C7980E94A10DE2E0F0E00E946A
:101AE000382CDE98C49A0E94CA2C84E690E00E94AA
:101AF000DE2CA8957091CF007F7B7093CF00E0E63D
:101B0000F0E0FA93EA930E94092122960091600086
:101B1000003011F40C949C0D7091CF0070647093A0
:101B2000CF0084E690E00E94DE2CDE9A6E98C49886
:101B3000C598C7980C949E0D0E94FE130895AB980B
:101B40000895AB9A089581E00E94ED2C70916A008F
:101B50007F7E70936A000091C10041E00423A88158
:101B6000B9810C93A881B9810C91003011F40C94C7
:101B7000BE0D70916A00706170936A007091CF0021
:101B80007F777093CF000091C10042E00423A881C9
:101B9000B9810C93A881B9810C91003011F40C9497
:101BA000D60D7091CF0070687093CF0070916A006D
:101BB0007E7F70936A000091C10044E00423A881F5
:101BC000B9810C93A881B9810C91003011F40C9467
:101BD000EE0D70916A00716070936A0070916A00F6
:101BE0007D7F70936A000091C10048E00423A881C2
:101BF000B9810C93A881B9810C91003011F40C9437
:101C0000060E70916A00726070936A0070916A00AB
:101C10007F7D70936A000091C10040E20423A88197
:101C2000B9810C93A881B9810C91003011F40C9406
:101C30001E0E70916A00706270936A007091CF00FE
:101C40007F7E7093CF000091C20041E00423A88101
:101C5000B9810C93A881B9810C91003011F40C94D6
:101C6000360E7091CF0070617093CF000091C2006A
:101C700046E00423A881B9810C93A881B9810C9115
:101C800042E00E94F32D0C93A881B9818C9180933E
:101C9000D0000091D000033011F00C94520E82E07D
:101CA0008093D00081E0481A8827580A2296089528
:101CB00082E00E94ED2C81E00E94ED2C81E00E94E8
:101CC000ED2C80E0AA81BB818C9383E4ACE9B0E089
:101CD0008C938FE4ADE9B0E08C938EE4AEE9B0E094
:101CE0008C9386E4AFE9B0E08C9389E4A0EAB0E09D
:101CF0008C93AAE6B0E08C9185FBA881B9818827F6
:101D000080F98C9370916A00706270936A00A2E708
:101D1000B0E00D911D912D913C91A2E9B0E00D93A1
:101D20001D932D933C935A924A92A2E9B0E00D91F3
:101D30001D912D913C91A42DB52D0D931D932D93A7
:101D40003C9384E00E94792B5A924A9280E090E082
:101D5000A42DB52D8D939C9382E00E94792B5A92ED
:101D60004A9281E0A42DB52D8C9381E00E94792BBD
:101D70000E940D15269687E00E94752B8FE00E9429
:101D8000ED2CE4EAF0E006E0A881B9810E94CA2DBA
:101D9000A881B981E8E9FCE50E94032E0FB68FE027
:101DA000481A8827580A22960FBE81E009F080E081
:101DB0008F9300918D00003181E009F080E09F91C8
:101DC0008923882311F40C94330F81E0AA81BB810D
:101DD0008C93A2E9B0E00D911D912D913C91A2E769
:101DE000B0E00D931D932D933C9370916A007F7D1D
:101DF00070936A005A924A92A2E9B0E00D911D9147
:101E00002D913C91A42DB52D0D931D932D933C93B5
:101E100084E00E94792B5A924A9280E090E0A42DAF
:101E2000B52D8D939C9382E00E94792B5A924A9211
:101E300080E0A42DB52D8C9381E00E94792B0E9427
:101E40000D15269687E00E94752BA2E9B0E00D9152
:101E50001D912D913C91A2E7B0E00D931D932D9320
:101E60003C930E948D0FA881B9818C9180FBAAE6DA
:101E7000B0E08C9185F98C93A6E7B0E00D911D91AF
:101E80002D913C91A2E7B0E00D931D932D933C93CF
:101E9000A2E7B0E00D911D912D913C91A2E9B0E037
:101EA0000D931D932D933C935A924A92A2E9B0E070
:101EB0000D911D912D913C91A42DB52D0D931D9348
:101EC0002D933C9384E00E94792B5A924A9280E0B1
:101ED00090E0A42DB52D8D939C9382E00E94792BE8
:101EE0005A924A9280E0A42DB52D8C9381E00E94F5
:101EF000792B0E940D15269687E00E94752BAA81EA
:101F0000BB818C91AE81BF818D9388278C9384E0B7
:101F1000481A8827580A2696089582E00E94ED2CD8
:101F200081E00E94ED2C81E00E94ED2C789481E00C
:101F300090E0AC81BD818D939C93EA81FB81FA9303
:101F4000EA93EE81FF81FA93EA930E94A31124960B
:101F5000AA81BB810C91013011F00C94BA0F82E080
:101F600090E0AC81BD818D939C9381E08093C10012
:101F70000C94D60F023011F00C94C90F83E090E05E
:101F8000AC81BD818D939C9380E08093C1000C94C3
:101F9000D60F033011F00C94D60F84E090E0AC81A2
:101FA000BD818D939C9383E08093C100EEE0F0E0CF
:101FB000A1ECB0E07BE70E94D82DEC81FD81FA9383
:101FC000EA935A924A9280E0A42DB52D8C9381E039
:101FD0000E94792B0E94E011249681E00E94752BCB
:101FE0000091CE00003011F00C94F00F88EC90E0DE
:101FF0000E94DE2C85E090E0AC81BD818D939C93A6
:10200000EA81FB81FA93EA93EE81FF81FA93EA93E6
:102010000E94A3112496EEE0F0E0A1ECB0E00E9453
:10202000E92DAA81BB810C91033011F00C941A1098
:102030000C94B710AA81BB810C91013011F00C9463
:102040002810A1ECB0E08C9188608C930C94311036
:10205000023011F00C943110A1ECB0E08C91877F2C
:102060008C93EEE0F0E0A1ECB0E07BE70E94D82D8D
:1020700088EC90E00E94DE2C86E090E0AC81BD818F
:102080008D939C93EA81FB81FA93EA93EE81FF8121
:10209000FA93EA930E94A3112496AA81BB810C9122
:1020A000033011F00C9456100C94B710EEE0F0E0F1
:1020B000A1ECB0E00E94E92DAA81BB810C91013016
:1020C00011F00C946A10A1ECB0E08C9184608C93B8
:1020D0000C947310023011F00C947310A1ECB0E06A
:1020E0008C918B7F8C93EEE0F0E0A1ECB0E07BE78D
:1020F0000E94D82D88EC90E00E94DE2C87E090E0D2
:10210000AC81BD818D939C93EA81FB81FA93EA9324
:10211000EE81FF81FA93EA930E94A3112496EEE0E8
:10212000F0E0A1ECB0E00E94E92DAA81BB810C9106
:10213000013011F00C94A310A1ECB0E08C918062FE
:102140008C930C94AC10023011F00C94AC10A1ECF8
:10215000B0E08C918F7D8C93EEE0F0E0A1ECB0E0EC
:102160007BE70E94D82D88EC90E00E94DE2C88E06E
:1021700090E0AC81BD818D939C93EC81FD81FA93BD
:10218000EA930E94811122960091C10043E004234A
:10219000A881B9810C93A881B9810C91003011F00C
:1021A0000C94DA1083E090E0AC81BD818D939C9318
:1021B0000C94F010013011F00C94E61082E090E0E5
:1021C000AC81BD818D939C930C94F010033011F081
:1021D0000C94F01084E090E0AC81BD818D939C93D1
:1021E000EC81FD81FA93EA930E948111229600917D
:1021F000C10048E00423A881B9810C93A881B9816A
:102200000C91003011F00C940D118AE090E0AC813B
:10221000BD818D939C930C941711083011F00C9490
:10222000171189E090E0AC81BD818D939C93EC8186
:10223000FD81FA93EA930E94811122960091C100D8
:1022400044E00423A881B9810C93A881B9810C9141
:10225000003011F00C9434118BE090E0AC81BD8122
:102260008D939C930C943E11043011F00C943E110C
:102270008CE090E0AC81BD818D939C93EC81FD81DD
:10228000FA93EA930E94811122960091C10040E2E4
:102290000423A881B9810C93A881B9810C910030E5
:1022A00011F00C945B118DE090E0AC81BD818D93B9
:1022B0009C930C946511003211F00C9465118EE022
:1022C00090E0AC81BD818D939C93EC81FD81FA936C
:1022D000EA930E94811122968FE090E0AC81BD814B
:1022E0008D939C93EC81FD81FA93EA930E94811176
:1022F00022960E94A30D84E0481A8827580A269641
:102300000895E881F981FA93EA935A924A9280E01B
:10231000A42DB52D8C9381E00E94792B0E94E011B1
:10232000249681E00E94752B82E390E00E94DE2CCF
:102330000091CE00003011F00C94981182E390E0EF
:102340000E94DE2C089581E00E94ED2CEA81FB8141
:10235000FA93EA935A924A9280E0A42DB52D8C9379
:1023600081E00E94792B0E94E011249681E00E9476
:10237000752B84E690E00E94DE2CE881F981FA93C7
:10238000EA930E94C11C2296A881B9810C91003069
:1023900018F011F00C94CE110C94BD110E94570D41
:1023A00084E190E00E94DE2CA881B9818C91AC81FF
:1023B000BD818C9381E0481A8827580A2296089597
:1023C00082E00E94ED2C81E00E94ED2C8EB5887F8A
:1023D0008EBD70916A00777F70936A00A2E7B0E0CB
:1023E0000D911D912D913C91A2E9B0E00D931D93AB
:1023F0002D933C935A924A92A2E9B0E00D911D911F
:102400002D913C91A42DB52D0D931D932D933C93AF
:1024100084E00E94792B5A924A92AA85BB858D91BD
:102420009C91A42DB52D8D939C9382E00E94792BD5
:102430005A924A9280E0A42DB52D8C9381E00E949F
:10244000792B0E940D15269687E00E94752B40E09F
:1024500050E060E070E0AEE8B0E00D911D912D918C
:102460003C910E944F2D11F00C9438120C94F813EB
:102470000E94AB275A924A928091BB00A42DB52DA1
:102480008C9381E00E94792B0E94F727229681E0AD
:102490000E94752B5A924A92ACEBB0E08D919C91C0
:1024A000A42DB52D8D939C9382E00E94792B0E94E0
:1024B0008F28229682E00E94752B0027AFECB0E0B7
:1024C0008C9184FB0EF401E041E0041711F00C94B0
:1024D00083125A924A928091BE00A42DB52D8C93FE
:1024E00081E00E94792B5A924A928091BF00A42DDC
:1024F000B52D8C9381E00E94792B0E945028249660
:1025000082E00E94752BA2E9B0E00D911D912D9102
:102510003C91A1EDB0E00D931D932D933C93A2E966
:10252000B0E00D911D912D913C91AEE8B0E04D9140
:102530005D916D917C910E94452DA5EDB0E00D93CC
:102540001D932D933D9380E0A881B9818C930E94C7
:102550003D2481E090E0AA81BB818D939C93AA8168
:10256000BB810D911C910F3F51E0150718F011F040
:102570000C94E912AA81BB81AD90BC90A9EDB0E0AA
:10258000AA0DBB1D0C910F3F81E009F080E08F93F5
:10259000AA81BB81AD90BC90AAEDB0E0AA0DBB1D95
:1025A0000C910F3E80E010F009F081E09F918923AB
:1025B000882311F40C94E21281E0A881B9818C93F4
:1025C0000C94E912AA81BB810E948C2B11F00C940F
:1025D000AF12A881B9810C91013011F00C94A712AF
:1025E000AA81BB81AD90BC90ABEDB0E0AA0DBB1D44
:1025F0008C91AA81BB818D9388278C93AA81BB8102
:102600000D911C9140E150E00E94BE2BAA81BB813C
:102610004D935C9380E18093C300AA81BB810D91AF
:102620001C91013050E0150711F00C941C1384E04C
:102630008093C3000C94A913023050E0150711F0E9
:102640000C94271385E08093C3000C94A9130330E6
:1026500050E0150711F00C94321386E08093C3000C
:102660000C94A913043050E0150711F00C943D139D
:1026700087E08093C3000C94A913053050E0150740
:1026800011F00C94481388E08093C3000C94A913B4
:10269000063050E0150711F00C9453138AE0809334
:1026A000C3000C94A913073050E0150711F00C94E7
:1026B0005E138CE08093C3000C94A913083050E0A3
:1026C000150711F00C9469138EE08093C3000C94ED
:1026D000A913093050E0150711F00C94741380E130
:1026E0008093C3000C94A9130A3050E0150711F031
:1026F0000C947F1384E18093C3000C94A9130B30D6
:1027000050E0150711F00C948A1388E18093C30000
:102710000C94A9130C3050E0150711F00C9495138C
:102720008CE18093C3000C94A9130D3050E0150781
:1027300011F00C94A01380E28093C3000C94A913B1
:102740000E3050E0150711F00C94A91388E2809325
:10275000C300AEE8B0E00D911D912D913C9140E099
:1027600052E060E070E00E943E2CA5E6B0E00D93E0
:102770001D932D933D93A5E6B0E00D911D912D91F4
:102780003C91A3ECB0E04C915527662777270E9437
:10279000432CA5E6B0E04D935D936D937D93A5E644
:1027A000B0E00D911D912D913C9148EE53E060E019
:1027B00070E00E94432CA5E6B0E04D935D936D93CD
:1027C0007D93AC81BD810C91003011F00C94F81315
:1027D00081E08093CE0088EC9FEA9DBD8CBD89B7D7
:1027E000846089BF81E08EBD85E090E00E94DE2C90
:1027F00083E0481A8827580A24960895A895A2E7E6
:10280000B0E00D911D912D913C91A6E7B0E00D93A4
:102810001D932D933C93A2E7B0E00D911D912D9156
:102820003C91A2E9B0E00D931D932D933C935A92F5
:102830004A92A2E9B0E00D911D912D913C91A42DF9
:10284000B52D0D931D932D933C9384E00E94792B1D
:102850005A924A9280E090E0A42DB52D8D939C93DE
:1028600082E00E94792B5A924A9280E0A42DB52DE5
:102870008C9381E00E94792B0E940D15269687E0AB
:102880000E94752BA895A2EBB0E00D911C91013030
:1028900050E0150710F00C9474145A924A9281E09B
:1028A000A42DB52D8C9381E00E94792B0E94E928FC
:1028B000229681E00E94752B8CE291E00E94DE2C32
:1028C0005A924A9280E0A42DB52D8C9381E00E940B
:1028D000792B0E94E928229681E00E94752B709145
:1028E000CF0070647093CF00A895A2E7B0E00D917F
:1028F0001D912D913C91A2E9B0E00D931D932D9374
:102900003C93A6EBB0E00D911C91003050E0150710
:1029100081E009F080E08F93A2EBB0E04D915C91F3
:10292000A6EBB0E00D911C910417150780E010F0A4
:1029300009F081E09F91892B882311F40C94A6144F
:1029400081E090E0A6EBB0E08D939C930E94A10DF6
:10295000089584E00E94ED2CA1EDB0E00D911D9151
:102960002D913C91A881B9810D931D932D933C939A
:10297000A2E7B0E00D911D912D913C91A2E9B0E04C
:102980000D931D932D933C935A924A92A2E9B0E085
:102990000D911D912D913C91A42DB52D0D931D935D
:1029A0002D933C9384E00E94792B5A924A928FE1B6
:1029B0009EE4A42DB52D8D939C9382E00E94792BEB
:1029C0005A924A9280E0A42DB52D8C9381E00E940A
:1029D000792B0E940D15269687E00E94752BA2E7A1
:1029E000B0E00D911D912D913C91A2E9B0E00D93C5
:1029F0001D932D933C93A881B9810D911D912D912B
:102A00003C91A1EDB0E00D931D932D933C9384E098
:102A1000481A8827580A2296089581E00E94ED2CD2
:102A200081E00E94ED2C81E00E94ED2C80E090E09E
:102A3000A4EBB0E08D939C9370916A007F7B7093C0
:102A40006A0000E010E020E030E0AEE8B0E00D9376
:102A50001D932D933C930027AAE6B0E08C9185FB53
:102A60000EF401E041E0041781E009F080E08F936B
:102A7000A885B9850D911C91003050E0150781E0C3
:102A800009F480E09F9189238F93AE81BF810C91DF
:102A9000003081E009F080E09F918923882311F4C0
:102AA0000C94AD15A6E9B0E0E885F9850E94622D89
:102AB000E6E9F0E0A8E6B7E00E94BE2DE8E6F7E020
:102AC000A6E9B0E01127222704E033270E94072D52
:102AD00081E4AC81BD818C93AC81BD818C9180936C
:102AE0009C0081E0E6E9F0E001E00A93ABE6B0E0AB
:102AF0000E94C32DABE6B0E08C91ADE9B0E08C93C1
:102B000082E0E6E9F0E001E00A93ABE6B0E00E9483
:102B1000C32DABE6B0E08C91AEE9B0E08C9383E0DE
:102B2000E6E9F0E001E00A93ABE6B0E00E94C32DD5
:102B3000ABE6B0E08C91AFE9B0E08C9384E0E6E9DD
:102B4000F0E001E00A93ABE6B0E00E94C32DABE6F3
:102B5000B0E08C91A0EAB0E08C9389B78B7F89BFFD
:102B60008EB5887F8EBD81B5886181BD877F81BD2F
:102B7000AAECB0E00D911D912D913C91A6ECB0E036
:102B80000D931D932D933C93A6E7B0E04D915D917D
:102B90006D917C91A2E7B0E00D911D912D913C913A
:102BA0000E944F2D11F00C94DF1502E010E020E0A0
:102BB00030E0A6ECB0E00D931D932D933C9380E0A4
:102BC000A881B9818C93EA81FB81FA93EA935A92A6
:102BD0004A92AE85BF850D911D912D913C91A42DFA
:102BE000B52D0D931D932D933C9384E00E94792B7A
:102BF0000E943426249684E00E94752BAA81BB8112
:102C00000C910E3F11F40C9411167091CF0070646A
:102C10007093CF0070916A00706470936A000C9496
:102C200024165A924A92AA85BB858D919C91A42D17
:102C3000B52D8D939C9382E00E94792B0E942517DD
:102C4000229682E00E94752BA881B9818C918F5FBA
:102C50008C9340916F00A881B9810C91041781E099
:102C600009F080E08F930027AAE6B0E08C9186FB04
:102C70000EF401E041E0041781E009F480E09F9147
:102C80008923882311F40C94DA1600917E000B300E
:102C900011F00C948716E6ECF0E0FA93EA935A925E
:102CA0004A92A6ECB0E00D911D912D913C91A42D7E
:102CB000B52D0D931D932D933C9384E00E94792BA9
:102CC0000E94651B249684E00E94752BEA85FB8593
:102CD000FA93EA935A924A92A6ECB0E00D911D91B4
:102CE0002D913C91A42DB52D0D931D932D933C93C7
:102CF00084E00E94792B0E94FB1A249684E00E94B3
:102D0000752B80E0A881B9818C930C94D816A6E726
:102D1000B0E04D915D916D917C91A2E7B0E00D9195
:102D20001D912D913C910E944F2D11F00C949E16F7
:102D3000AA85BB850E947D2B0C94D816E6ECF0E0AA
:102D4000FA93EA935A924A92A6ECB0E00D911D9143
:102D50002D913C91A42DB52D0D931D932D933C9356
:102D600084E00E94792B0E94651B249684E00E94D7
:102D7000752BEA85FB85FA93EA935A924A92A6EC60
:102D8000B0E00D911D912D913C91A42DB52D0D9389
:102D90001D932D933C9384E00E94792B0E94FB1A93
:102DA000249684E00E94752B80E0A881B9818C93E1
:102DB0000C94DE16AA85BB850E947D2B0027AAE60F
:102DC000B0E08C9186FB0EF401E041E0041711F0B5
:102DD0000C94E315C49AA885B9850D911C91003017
:102DE00050E0150711F00C94FD16A4EBB0E08D91A6
:102DF0009C91A2EBB0E08D939C930091CE000130AA
:102E000081E009F080E08F930027AFECB0E08C9177
:102E100086FB0EF401E040E0041781E009F080E059
:102E20009F918923882311F40C941F1780E593EC5C
:102E30009DBD8CBD81E08EBD89B7846089BF83E074
:102E4000481A8827580A2696089584E00E94ED2C97
:102E500084E00E94ED2C81E00E94ED2C81E00E9434
:102E6000ED2C81E00E94ED2C81E00E94ED2C80E0B1
:102E7000AE81BF818C93AE81BF810C910F3018F071
:102E800011F00C94081981E0AC81BD818C93AC8168
:102E9000BD810C910C3018F011F00C9467178FEF76
:102EA0000E94D12C0E94D32C0E94D22CAC81BD81D7
:102EB000AD90BB24A0E8B0E0AA0DBB1D8C93AC8103
:102EC000BD818C918F5F8C9311F00C9447178DE02E
:102ED000AC81BD818C93AC81BD810C91043118F023
:102EE00011F00C9485178FEF0E94D12C0E94D32CE7
:102EF0000E94D22CA881B9818C93AC81BD818C9128
:102F00008F5F8C9311F00C946B17EA85FB85FA9315
:102F1000EA93EA85FB85FA93EA930E949019249636
:102F20000027AAE6B0E08C9186FB0EF401E041E0B8
:102F3000041711F00C949E170C94001980E0AA81DC
:102F4000BB818C9300918C00003281E009F080E01D
:102F50008F9300918C00003181E009F080E09F9117
:102F6000892B882311F40C94B91781E0AA81BB81C5
:102F70008C9300918100003081E009F480E08F9310
:102F800000918100053E81E009F480E09F91892352
:102F90008F93AA81BB810C91013081E009F080E020
:102FA0009F918923882311F40C94F51800918C00CB
:102FB000003211F00C94E017A4EBB0E00E948C2BCF
:102FC0000027AAE6B0E08C9185FB0EF401E040E01A
:102FD000041711F00C94151881E0AC81BD818C931D
:102FE000AC85BD854D915C91A4EBB0E00D911C9139
:102FF0000417150781E009F080E08F93A4EBB0E09F
:103000000D911C91003050E0150780E010F009F0A0
:1030100081E09F918923882311F40C94131880E098
:10302000AC81BD818C930C94491880E0AC81BD814A
:103030008C9381E0A881B9818C93A881B9810C918E
:10304000053018F011F00C944918A881B981AD90A1
:10305000BB24ABE9B0E0AA0DBB1D4C91A881B9819E
:10306000AD90BB24A0E8B0E0AA0DBB1D0C910417E5
:1030700011F40C94411881E0AC81BD818C930C94C7
:103080004918A881B9818C918F5F8C9311F00C94B1
:103090001D18AC81BD810C91003081E009F080E009
:1030A0008F93AC85BD850D911C910F315EE41507A2
:1030B00081E009F080E09F91892B882311F40C9422
:1030C000F5180E942219A885B9850D911D912D91A1
:1030D0003C9140E052E060E070E00E94432CAEE89A
:1030E000B0E04D935D936D937D93E2E9F0E0FA9348
:1030F000EA935A924A92AE85BF850D911D912D910A
:103100003C91A42DB52D0D931D932D933C9384E0FC
:103110000E94792B0E94FB1A249684E00E94752B52
:1031200080918C0080938D00AC85BD850D911C91A4
:103130000F315EE4150711F00C94C618A8E6B7E04D
:10314000E4EBF0E00E94622D0E941D2CE0EAFCE519
:103150000E94252CA4EAB0E00E941F2CE0EAFCE5C6
:103160000E94252C00918C00003111F00C94BC18A9
:10317000E2EAFCE50E94252CA8E6B7E0E885F9859F
:103180000E94652D0E941D2C0E94312CAC81BD81B6
:103190000C91003011F00C94F51870916A00706475
:1031A00070936A0000918D00003181E009F080E0A9
:1031B0008F93AC85BD850D911C910F315EE4150791
:1031C00081E009F480E09F918923882311F40C9415
:1031D000F518AA85BB850D911D912D913C91AAEC06
:1031E000B0E00D931D932D933C930091810000302E
:1031F00011F00C94001970916A00706470936A0069
:10320000AE81BF818C918F5F8C9311F00C943B1732
:103210008FEF0E94D12C0E94D32C0E94D22CA0E6CA
:10322000B0E08C938FEF0E94D12C0E94D32C0E948F
:10323000D22CA0E6B0E08C938CE0481A8827580A7C
:103240002C96089581E00E94ED2CA4EAB0E0882736
:103250008C9381E0A881B9818C93A881B9810C916C
:10326000083018F011F00C945C19A881B981AD9068
:10327000BB24A0E8B0E0AA0DBB1D0C91003211F4F4
:103280000C945419A881B981AD90BB24A0E8B0E09A
:10329000AA0DBB1D8C91A4EAB0E08F930E940A2C6A
:1032A0008F918D9388278C93A881B9818C918F5FA2
:1032B0008C9311F00C942D19A4EAB0E00E940A2C12
:1032C000E6EAFCE50E94042C89E0A881B9818C9390
:1032D000A881B9810C910B3018F011F00C948A1967
:1032E000A881B981AD90BB24A0E8B0E0AA0DBB1DB8
:1032F0008C91A4EAB0E08F930E940A2C8F918D9359
:1033000088278C93A881B9818C918F5F8C9311F061
:103310000C94681981E0481A8827580A2296089563
:1033200081E00E94ED2C81E00E94ED2C84E00E945F
:10333000ED2C8FEF0E94D12C0E94D32C0E94D22C16
:10334000AC81BD818C938FEF0E94D12C0E94D32C35
:103350000E94D22CAA81BB818C93AA81BB810C9143
:1033600011272227332740E051E060E070E00E94FF
:103370003E2CA885B9850D931D932D933D93A8856B
:10338000B9850D911D912D913C91AC81BD814C91E0
:103390005527662777270E94452DA885B9850D9367
:1033A0001D932D933D93A885B9850D911D912D9168
:1033B0003C9140E050E061E070E00E943E2CA8812A
:1033C000B9810D931D932D933D938FEF0E94D12CC6
:1033D0000E94D32C0E94D22CAC81BD818C938FEFA4
:1033E0000E94D12C0E94D32C0E94D22CAC81BD8192
:1033F0008C938FEF0E94D12C0E94D32C0E94D22C50
:10340000AC81BD818C938FEF0E94D12C0E94D32C74
:103410000E94D22CAC81BD818C938FEF0E94D12C65
:103420000E94D32C0E94D22CAC81BD818C938FEF53
:103430000E94D12C0E94D32C0E94D22CAA81BB8145
:103440008C93AA81BB810C9111272227332740E05E
:1034500051E060E070E00E943E2CA885B9850D9394
:103460001D932D933D93A885B9850D911D912D91A7
:103470003C91AC81BD814C915527662777270E94EE
:10348000452DA885B9850D931D932D933D93A88552
:10349000B9850D911D912D913C91A881B9814D91D6
:1034A0005D916D917C910E94452DA885B9850D9304
:1034B0001D932D933D938FEF0E94D12C0E94D32C0E
:1034C0000E94D22CAC81BD818C938FEF0E94D12CB5
:1034D0000E94D32C0E94D22CAA81BB818C93AA81FA
:1034E000BB810C9111272227332740E051E060E097
:1034F00070E00E943E2CA881B9810D931D932D93FD
:103500003D93A881B9810D911D912D913C91AC8184
:10351000BD814C915527662777270E94452DA881AC
:10352000B9810D931D932D933D938FEF0E94D12C64
:103530000E94D32C0E94D22CAC81BD818C938FEF42
:103540000E94D12C0E94D32C0E94D22CAA81BB8134
:103550008C93AA81BB810C9111272227332740E04D
:1035600051E060E070E00E943E2CAE81BF810D937F
:103570001D932D933D93AE81BF810D911D912D9192
:103580003C91AC81BD814C915527662777270E94DD
:10359000452DAE81BF810D931D932D933D93AE813B
:1035A000BF810D911D912D913C9140E050E061E073
:1035B00070E00E943E2CAE81BF810D931D932D9330
:1035C0003D93AE81BF810D911D912D913C91A881BC
:1035D000B9814D915D916D917C910E94452DAE8197
:1035E000BF810D931D932D933D9386E0481A882744
:1035F000580A2696089584E00E94ED2C84E00E94EB
:10360000ED2CAC81BD810D911D912D913C9142E03D
:1036100050E060E070E00E944A2DA881B9810D93CE
:103620001D932D933D93AFE6B0E00C911127222717
:103630003327A881B9814D915D916D917C910E9454
:103640003E2CAA81BB810D931D932D933D93AA819E
:10365000BB810D911D912D913C91A6E7B0E04D915C
:103660005D916D917C910E94452DAA81BB810D9346
:103670001D932D933D9300917E000B3011F40C941B
:10368000531BAA81BB810D911D912D913C9140E26C
:1036900050E060E070E00E94452DAA81BB810D934F
:1036A0001D932D933D93AA81BB810D911D912D9169
:1036B0003C91AE81BF810D931D932D933C9388E087
:1036C000481A8827580A2496089584E00E94ED2C11
:1036D00082E00E94ED2C00917E000B3011F00C94E2
:1036E000A91BAC81BD810D911D912D913C9140E8AC
:1036F00050E060E070E00E94432CA1EDB0E04D93FB
:103700005D936D937D93AC81BD810D911C9140E8DB
:1037100050E00E94DE2BA881B9810D931C93A881F3
:10372000B9810D911C9144E050E00E94F82BA881D2
:10373000B9810D931C93A881B9810D911C9144E02E
:1037400050E0040F151FA881B9810D931C930C94B0
:10375000DF1BAC81BD810D911D912D913C9140E00D
:1037600051E060E070E00E94432CA1EDB0E04D9389
:103770005D936D937D93AC81BD810D911C9140E073
:1037800051E00E94DE2BA881B9810D931C93A88182
:10379000B9810D911C9142E050E00E94F82BA88164
:1037A000B9810D931C93A881B9810D911C9142E0C0
:1037B00050E0040F151FA881B9810D931C93A1ED52
:1037C000B0E00D911D912D913C91AAE7B0E04D9193
:1037D0005D916D917C910E94452DA1EDB0E00D931E
:1037E0001D932D933D93A1EDB0E00D911D912D9171
:1037F0003C91ADE6B0E04D915C91662777270E9441
:10380000452DA1EDB0E00D931D932D933D930E94A6
:103810003D24A881B981AD90BC90A9EDB0E0AA0D7E
:10382000BB1D8C91AA81BB818D9388278D938D932D
:103830008C93A881B9810E94922BAA81BB810D91A2
:103840001D912D913C9140E051E060E070E00E94BC
:103850003E2CAA81BB810D931D932D933D93AA818C
:10386000BB810D911D912D913C91A881B981AD90A5
:10387000BC90A9EDB0E0AA0DBB1D4C915527662761
:1038800077270E94452DAA81BB810D931D932D930F
:103890003D9300917E000B3011F00C94AF1CA88179
:1038A000B9810E94922BAA81BB810D911D912D910E
:1038B0003C9140E051E060E070E00E943E2CAA8123
:1038C000BB810D931D932D933D93AA81BB810D91D7
:1038D0001D912D913C91A881B981AD90BC90A9ED2D
:1038E000B0E0AA0DBB1D4C915527662777270E9493
:1038F000452DAA81BB810D931D932D933D93A881E6
:10390000B9810E94922BAA81BB810D911D912D91AD
:103910003C9140E051E060E070E00E943E2CAA81C2
:10392000BB810D931D932D933D93AA81BB810D9176
:103930001D912D913C91A881B981AD90BC90A9EDCC
:10394000B0E0AA0DBB1D4C915527662777270E9432
:10395000452DAA81BB810D931D932D933D93AA8183
:10396000BB810D911D912D913C91AE81BF810D9335
:103970001D932D933C9386E0481A8827580A249675
:10398000089580E0A881B9818C930027BB27A0E32C
:103990008C9183FB0EF401E040E0041711F00C94CD
:1039A000D51C82E0A881B9818C930027BB27A0E3B6
:1039B0008C9184FB0EF401E040E0041711F00C94AC
:1039C000E51C81E0A881B9818C930027BB27A3E384
:1039D0008C9181FB0EF401E040E0041711F00C948F
:1039E000F51C83E0A881B9818C930027BB27A3E352
:1039F0008C9181FB0EF401E040E0041781E009F0B6
:103A000080E08F930027BB27A0E38C9183FB0EF40B
:103A100001E040E0041781E009F080E09F918923F4
:103A2000882311F40C94181D84E0A881B9818C932B
:103A3000089581E00E94ED2C81E00E94ED2C82E04F
:103A40000E94ED2C0027AFECB0E08C9183FB0EF4CC
:103A500001E041E0041711F00C94441D80E0AC81BA
:103A6000BD818C930027BB27A9E38C9185FB0EF4C5
:103A700001E040E0041711F00C94421D81E0AC819C
:103A8000BD818C930C94441E5398549880E081BB64
:103A9000909A919AEF93FF93E0EFF1E00E94B22C9D
:103AA000FF91EF9180E0AC81BD818C930027BB2713
:103AB000A0E38C9180FB0EF401E040E0041711F0CC
:103AC0000C94661D81E0AC81BD818C930027BB27DF
:103AD000A0E38C9181FB0EF401E040E0041711F0AB
:103AE0000C94771DAC81BD818C918E5F8C930027E7
:103AF000BB27A9E38C9185FB0EF401E040E004179D
:103B000011F00C94881DAC81BD818C918C5F8C93DD
:103B10000027BB27A9E38C9184FB0EF401E040E071
:103B2000041711F00C94991DAC81BD818C91885FB4
:103B30008C93AC81BD810C91003018F011F00C9485
:103B4000A31D0C94FC1D85E090E00E94DE2C80E01B
:103B5000AA81BB818C930027BB27A0E38C9180FBBB
:103B60000EF401E040E0041711F00C94BB1D81E05D
:103B7000AA81BB818C930027BB27A0E38C9181FB9A
:103B80000EF401E040E0041711F00C94CC1DAA8162
:103B9000BB818C918E5F8C930027BB27A9E38C910E
:103BA00085FB0EF401E040E0041711F00C94DD1DDC
:103BB000AA81BB818C918C5F8C930027BB27A9E3E2
:103BC0008C9184FB0EF401E040E0041711F00C949A
:103BD000EE1DAA81BB818C91885F8C93AA81BB81E9
:103BE0004C91AC81BD810C91041711F40C94FC1D17
:103BF00080E0AC81BD818C93AC81BD810C910330A0
:103C000011F00C94091E82E0AC81BD818C930C9460
:103C10003F1EAC81BD810C91043081E008F480E04E
:103C20008F93AC81BD810C91073081E010F009F0D9
:103C300080E09F918923882311F40C94251E83E052
:103C4000AC81BD818C930C943F1EAC81BD810C91E5
:103C5000083081E008F480E08F93AC81BD810C9145
:103C60000F3081E010F009F080E09F9189238823D4
:103C700011F40C943F1E84E0AC81BD818C9381E0F3
:103C800081BB9198539A549AAC81BD818C91AE813D
:103C9000BF818C9384E0481A8827580A2696089595
:103CA00081E00E94ED2C81E00E94ED2CAC81BD8171
:103CB0008C91A881B9818C930E949F0D88EC90E033
:103CC0000E94DE2C5A924A9281E0A42DB52D8C934D
:103CD00081E00E94792B0E94E928229681E00E94CF
:103CE000752BA895E9E6F0E0FA93EA930E94C11CCF
:103CF00022968AE090E00E94DE2C0091690000305C
:103D000011F00C94711E86E990E00E94DE2C5A920C
:103D10004A9280E0A42DB52D8C9381E00E94792BEE
:103D20000E94E928229681E00E94752B84E690E0AB
:103D30000E94DE2C5A924A9280E0A42DB52D8C93DD
:103D400081E00E94792B0E94E928229681E00E945E
:103D5000752BA895E9E6F0E0FA93EA930E94C11C5E
:103D600022960E94A10D5A924A9281E0A42DB52D6F
:103D70008C9381E00E94792B0E94E928229681E0B1
:103D80000E94752B84E690E00E94DE2C5A924A92A3
:103D900080E0A42DB52D8C9381E00E94792B0E94A8
:103DA000E928229681E00E94752B8AE090E00E942B
:103DB000DE2C5A924A9280E0A42DB52D8C9381E09E
:103DC0000E94792B0E94E928229681E00E94752B9F
:103DD0000E949F0D86E990E00E94DE2C0091690010
:103DE000003018F011F00C94F71E0C94A91E88E70F
:103DF00090E00E94DE2C5A924A9281E0A42DB52DCB
:103E00008C9381E00E94792B0E941820229681E0F9
:103E10000E94752BA881B9810C91023011F00C948D
:103E2000511F00916900013011F00C941C1F81E0BA
:103E30008093C1000C944A1F023011F00C94341F7F
:103E400080E08093C1005A924A9281E0A42DB52D62
:103E50008C9381E00E94792B0E941820229681E0A9
:103E60000E94752B0C944A1F033011F00C944A1FCA
:103E700083E08093C1005A924A9282E0A42DB52D2E
:103E80008C9381E00E94792B0E941820229681E079
:103E90000E94752BEEE0F0E0A1ECB0E07BE70E9421
:103EA000D82DA881B9810C91033011F00C94841F96
:103EB00000916900013011F00C94651FA2ECB0E094
:103EC0008C9181608C930C947D1F023011F00C94C6
:103ED0007D1FA2ECB0E08C918E7F8C935A924A9217
:103EE00081E0A42DB52D8C9381E00E94792B0E9456
:103EF0001820229681E00E94752BEFE0F0E0A2EC02
:103F0000B0E07BE70E94D82DA881B9810C910130E7
:103F100011F00C94D61F00916900013011F00C943F
:103F20009D1FA2ECB0E08C9182608C93A2ECB0E07B
:103F30008C918B7F8C930C94CF1F023011F00C94DA
:103F4000B71FA2ECB0E08C91897F8C935A924A9271
:103F500081E0A42DB52D8C9381E00E94792B0E94E5
:103F60001820229681E00E94752B0C94CF1F0330FD
:103F700011F00C94CF1FA2ECB0E08C9186608C9372
:103F80005A924A9282E0A42DB52D8C9381E00E9432
:103F9000792B0E941820229681E00E94752BEFE079
:103FA000F0E0A2ECB0E07BE70E94D82D0E94A30DC8
:103FB000A895E9E6F0E0FA93EA930E94C11C2296E4
:103FC00085E090E00E94DE2C00916900003011F045
:103FD0000C94D81F86E990E00E94DE2C5A924A92F7
:103FE00080E0A42DB52D8C9381E00E94792B0E9456
:103FF000E928229681E00E94752B86E990E00E94D4
:10400000DE2C5A924A9280E0A42DB52D8C9381E04B
:104010000E94792B0E94E928229681E00E94752B4C
:104020000E94A10D82E0481A8827580A2496089514
:1040300081E00E94ED2C81E0A881B9818C93AA8156
:10404000BB814C91A881B9810C91041718F011F033
:104050000C9445205A924A9282E0A42DB52D8C935F
:1040600081E00E94792B0E94E928229681E00E943B
:10407000752B8DE790E00E94DE2CA881B9818C9190
:104080008F5F8C9311F00C941F2081E0481A8827D1
:10409000580A2296089581E00E94ED2C81E0A881C3
:1040A000B9818C93A881B9810C91063018F011F078
:1040B0000C946E200E949F0D8FE090E00E94DE2CF9
:1040C0000E94A10D84E690E00E94DE2CA881B981B7
:1040D0008C918F5F8C9311F00C94522081E0481AE0
:1040E0008827580A229608950E94CA2CC39A88EC01
:1040F00090E00E94DE2C81B5886081BD0E94AB27D4
:104100005A924A9281E0A42DB52D8C9381E00E94B1
:10411000792B0E94F727229681E00E94752B81B5AA
:10412000886181BD877F81BD84E690E00E94DE2C9E
:10413000FF27E0E1FA93EA935A924A928BE0A42D8A
:10414000B52D8C9381E00E94792B0E947F2A2496C2
:1041500081E00E94752B013051E0150711F00C949D
:10416000CA205A924A92ACEBB0E08D919C91A42D5A
:10417000B52D8D939C9382E00E94792B0E948F280D
:10418000229682E00E94752BE8EAFCE50E94252C2D
:104190000E94312C5A924A9282E3A42DB52D8C9321
:1041A00081E00E94792B0E94F727229681E00E94ED
:1041B000752BC29AD89A82E390E00E94DE2C089573
:1041C00081E00E94ED2C81E00E94ED2C8FEFAA810E
:1041D000BB818C9380E0A881B9818C93A881B9813F
:1041E0000C91073018F011F00C94032191E0AA8192
:1041F000BB810E94C02CA881B9818C918F5F8C9368
:1042000011F00C94EE2082E0481A8827580A249670
:10421000089581E00E94ED2C81E00E94ED2C81E068
:104220000E94ED2C82E00E94ED2C82E00E94ED2C99
:104230008FEFAA85BB858C9381E0A885B9858C9387
:10424000A885B9850C91003418F011F00C94322136
:104250000E94E020A885B9858C918F5F8C9311F026
:104260000C942021C49881E0A885B9858C93A885F9
:10427000B9850C91003418F011F00C9449210E947A
:10428000E020A885B9858C918F5F8C9311F00C94F8
:1042900037218AE090E00E94DE2CA895EE81FF8114
:1042A000FA93EA935A924A9280E4A42DB52D8C9306
:1042B00081E00E94792B5A924A9200E010E020E0BF
:1042C00030E0A42DB52D0D931D932D933C9384E0E8
:1042D0000E94792B0E941A27269685E00E94752B52
:1042E000AE81BF810C91013011F40C948021C49AED
:1042F000ECEAFCE50E94252C0E94312C0C9437241A
:1043000081E0AA85BB858C93A89580E090E0A88188
:10431000B9818D939C93EE81FF81FA93EA935A922F
:104320004A9281E4A42DB52D8C9381E00E94792BD3
:104330005A924A9200E010E020E030E0A42DB52D22
:104340000D931D932D933C9384E00E94792B0E9442
:104350001A27269685E00E94752BA881B9810E94B4
:104360008C2BAE81BF810C91003081E009F080E0A0
:104370008F93A881B9810D911C91003050E01507F1
:1043800081E009F080E09F91892B882311F40C943F
:104390008B21C49AA881B9810D911C91003050E005
:1043A000150711F00C94DC21E4EBFCE50E94252CB0
:1043B0000E94312C0C943724A89584E690E00E944A
:1043C000DE2CA895C49881E090E00E94DE2CEE815E
:1043D000FF81FA93EA935A924A9280E5A42DB52D73
:1043E0008C9381E00E94792B5A924A9201E010E06E
:1043F00020E030E0A42DB52D0D931D932D933C931B
:1044000084E00E94792B0E941A27269685E00E945C
:10441000752B85E090E00E94DE2CC49A8AE090E043
:104420000E94DE2CA89500E010E020E030E0AAE732
:10443000B0E00D931D932D933C9300E010E020E03D
:1044400030E0A1EDB0E00D931D932D933C930E94BD
:104450003D2400E010E020E030E0A1EDB0E00D935D
:104460001D932D933C930027AFECB0E08C9186FB1D
:104470000EF401E041E0041711F00C9441220C9479
:104480003724A8950091E600023011F40C94D5224F
:1044900080919C0280937E00A3EAB2E00D911127E7
:1044A00040E051E00E94F82BAA81BB810D931C9340
:1044B000AA81BB810D911C91A2EAB2E04D915527D2
:1044C000040F151FAA81BB810D931C93AA81BB8188
:1044D0000D911C912227332740E050E061E070E00D
:1044E0000E943E2CAAE7B0E00D931D932D933D93BF
:1044F000A1EAB2E00D91112740E051E00E94F82BB3
:10450000AA81BB810D931C93AA81BB810D911C9143
:10451000A0EAB2E04D915527040F151FAA81BB8177
:104520000D931C93AAE7B0E00D911D912D913C9144
:10453000AA81BB814D915C91662777270E94452D0A
:10454000AAE7B0E00D931D932D933D9300917E005B
:104550000C3011F00C94AF228BE080937E00009120
:104560007E000E3011F00C94B8228BE080937E0018
:1045700000917E000F3011F00C94C1228BE08093EB
:104580007E00AAE7B0E00D911D912D913C91A1ED27
:10459000B0E00D931D932D933C930E943D24A1ED1B
:1045A000B0E00E94982B0C9429230091100106344E
:1045B00011F00C94FF2284E080937E0087E3A885AD
:1045C000B9858C93A885B9850C910C3318F011F03E
:1045D0000C94FD22A885B985AD90BB24A9EDB0E06F
:1045E000AA0DBB1D8C910E94342CA885B9858C9195
:1045F0008F5F8C9311F00C94E2220E94312C009179
:104600002C01063411F00C9429238BE080937E005A
:1046100083E5A885B9858C93A885B9850C91073564
:1046200018F011F00C942723A885B985AD90BB2410
:10463000A9EDB0E0AA0DBB1D8C910E94342CA88579
:10464000B9858C918F5F8C9311F00C940C230E9490
:10465000312CEEEBFCE50E94252CA8E6B7E0EEE756
:10466000F0E00E94712D0E941D2C0E94312CE0ED83
:10467000FCE50E94252CA8E6B7E0EAE7F0E00E94FE
:10468000652D0E941D2C0E94312C84E0A885B985DF
:104690008C93A885B9850C910B3018F011F00C940F
:1046A0006423A885B985AD90BB24A9EDB0E0AA0D1F
:1046B000BB1D8C910E94342CA885B9858C918F5F8D
:1046C0008C9311F00C9449230E94312C8091E700C7
:1046D00080936F00E2EEFCE50E94252CA8E6B7E08F
:1046E000EFE6F0E00E94712D0E941D2C0E94312CFB
:1046F00000916F00003011F00C9480230C9437244B
:1047000000916F00003418F011F00C9489230C9480
:104710008B230C9437248091E800AE81BF818C9369
:104720008091E900AC81BD818C93AC81BD819C916D
:10473000AE81BF818C91ADE6B0E08D939C9380916A
:10474000F000AE81BF818C938091F100AC81BD817E
:104750008C93AC81BD819C91AE81BF818C91A0E78F
:10476000B0E08D939C93A0E7B0E00D911C910030D8
:1047700050E0150711F00C94D3238091FE00AE8118
:10478000BF818C938091FF00AC81BD818C93AC8103
:10479000BD819C91AE81BF818C91A0E7B0E08D93EB
:1047A0009C930C94D323A0E7B0E00D911C910030B2
:1047B00050E0150711F00C94DF230C94372402E02D
:1047C00010E020E030E0A0E7B0E04D915C9166277A
:1047D00077270E943E2CA2E7B0E00D931D932D9306
:1047E0003D93A2E7B0E00D911D912D913C91ADE676
:1047F000B0E04D915C91662777270E94452DA2E796
:10480000B0E00D931D932D933D93A2E7B0E00D9181
:104810001D912D913C91A1EDB0E04D915D916D9177
:104820007C910E94452DA2E7B0E00D931D932D933E
:104830003D93E2EFFCE50E94252CA8E6B7E0E2E715
:10484000F0E00E94652D0E941D2C0E94312CA2E7F1
:10485000B0E00D911D912D913C91A1EDB0E00D9333
:104860001D932D933C9380E0AA85BB858C9387E0B4
:10487000481A8827580A2A96089581E00E94ED2C4C
:1048800081E00E94ED2C82E00E94ED2C82E00E94EB
:10489000ED2C8FEFAE81BF818C9391E0AE81BF8113
:1048A0000E94C02C91E0AE81BF810E94C02C91E09B
:1048B000AE81BF810E94C02C91E0AE81BF810E9479
:1048C000C02C91E0AE81BF810E94C02C91E0AE81EE
:1048D000BF810E94C02C91E0AE81BF810E94C02C9C
:1048E00091E0AE81BF810E94C02C91E0AE81BF817A
:1048F0000E94C02C91E0AE81BF810E94C02C91E04B
:10490000AE81BF810E94C02C91E0AE81BF810E9428
:10491000C02C91E0AE81BF810E94C02C91E0AE819D
:10492000BF810E94C02C91E0AE81BF810E94C02C4B
:1049300091E0AE81BF810E94C02CC49880E090E0DD
:10494000A881B9818D939C938FEF0E94D12C0E94F6
:10495000D32C0E94D22CAE81BF818C93A881B981C7
:104960000E948C2BAE81BF810C91003081E009F454
:1049700080E08F93A881B9810D911C91003050E0A7
:10498000150781E009F080E09F91892B882311F4BD
:104990000C94A424A881B9810D911C91003050E0A1
:1049A000150711F00C94E124EAEFFCE50E94252C98
:1049B0000E94312C7091CF0070647093CF000C94E2
:1049C0002E26EE81FF81FA93EA935A924A9281E56C
:1049D000A42DB52D8C9381E00E94792B5A924A9296
:1049E000A1EDB0E00D911D912D913C91A42DB52D1F
:1049F0000D931D932D933C9384E00E94792B0E948C
:104A00001A27269685E00E94752B0027AFECB0E0B0
:104A10008C9186FB0EF401E041E0041711F00C9438
:104A20002125E8E0FDE50E94252CA8E6B7E0E1EDB0
:104A3000F0E00E94652D0E941D2C0E94312C0C94E8
:104A40002E26A895AE81BF810C91003011F00C94F8
:104A50006C2580E090E0A881B9818D939C938FEFC5
:104A60000E94D12C0E94D32C0E94D22CAE81BF81F7
:104A70008C93A881B9810E948C2BAE81BF810C914F
:104A8000003081E009F480E08F93A881B9810D9115
:104A90001C91003050E0150781E009F080E09F9103
:104AA000892B882311F40C942F25A881B9810D91AD
:104AB0001C91003050E0150711F00C946C25E2E2D7
:104AC000FDE50E94252C0E94312C7091CF0070646E
:104AD0007093CF000C942E26AE81BF810C910F3FB6
:104AE00011F00C94B62580E090E0A881B9818D93F7
:104AF0009C938FEF0E94D12C0E94D32C0E94D22C29
:104B0000AE81BF818C93A881B9810E948C2BAE812C
:104B1000BF810C910F3F81E009F480E08F93A88161
:104B2000B9810D911C91003050E0150781E009F02A
:104B300080E09F91892B882311F40C947925A8811A
:104B4000B9810D911C91003050E0150711F00C94C3
:104B5000B625E0E3FDE50E94252C0E94312C7091E2
:104B6000CF0070647093CF000C942E26AE81BF816D
:104B70000C910E3F11F40C94D325EEE3FDE50E9459
:104B8000252CA8E6B7E0EE81FF810E94712D0E94DE
:104B90001D2C0E94312CC49A7091CF0070647093C8
:104BA000CF000C942E2680E090E0AA81BB818D93EB
:104BB0009C9380E0AE81BF818C93AE81BF810C91CC
:104BC0000F3F18F011F00C941526AA81BB810E94AA
:104BD0008C2B8FEF0E94D12C0E94D32C0E94D22CC0
:104BE000AA81BB81AD90BC90A9EDB0E0AA0DBB1D20
:104BF0008C93AA81BB810E948C2B8FEF0E94D12CB9
:104C00000E94D32C0E94D22CAA81BB81AD90BC9073
:104C1000A9EDB0E0AA0DBB1D8C93AE81BF818C9134
:104C20008F5F8C9311F00C94DD258FEF0E94D12CB7
:104C30000E94D32C0E94D22CAE81BF818C938FEF27
:104C40000E94D12C0E94D32C0E94D22CAE81BF8115
:104C50008C93C49AA1EDB0E00E947D2B86E0481AA7
:104C60008827580A2896089582E00E94ED2C81E05A
:104C70000E94ED2C80E0AE81BF818C930E94E020E9
:104C8000C49880E090E0AA81BB818D939C938FEFC4
:104C90000E94D12C0E94D32C0E94D22CA881B981D1
:104CA0008C93AA81BB810E948C2BA881B9810C9125
:104CB000003081E009F480E08F93AA81BB810D91DF
:104CC0001C91003050E0150781E009F080E09F91D1
:104CD000892B882311F40C944726AA81BB810D915E
:104CE0001C91003050E0150711F00C948426EAEF77
:104CF000FCE50E94252C0E94312C7091CF0070643D
:104D00007093CF000C941427E881F981FA93EA9309
:104D10005A924A9281E5A42DB52D8C9381E00E9490
:104D2000792B5A924A92AA85BB850D911D912D919E
:104D30003C91A42DB52D0D931D932D933C9384E0B0
:104D40000E94792B0E941A27269685E00E94752BD7
:104D5000A881B9810C91003011F00C94DB2680E021
:104D600090E0AA81BB818D939C938FEF0E94D12C00
:104D70000E94D32C0E94D22CA881B9818C93AA8145
:104D8000BB810E948C2BA881B9810C91003081E0FD
:104D900009F480E08F93AA81BB810D911C910030B2
:104DA00050E0150781E009F080E09F91892B88236E
:104DB00011F40C94B526A881B9810C910F3F11F024
:104DC0000C940E2780E090E0AA81BB818D939C9388
:104DD0008FEF0E94D12C0E94D32C0E94D22CA8814C
:104DE000B9818C93AA81BB810E948C2BA881B98147
:104DF0000C910F3F81E009F480E08F93AA81BB8181
:104E00000D911C91003050E0150781E009F080E021
:104E10009F91892B882311F40C94E826A881B981ED
:104E20008C91AE81BF818C9383E0481A8827580A01
:104E30002496089584E00E94ED2C81E00E94ED2CE0
:104E400082E00E94ED2C8FEFAA81BB818C9391E0D0
:104E5000AA81BB810E94C02C91E0A885B9850E94DF
:104E6000C02CAE81BF810D911D912D913C9140E0F0
:104E700052E060E070E00E943E2CAC81BD810D9359
:104E80001D932D933D93AC81BD818F9314968E918C
:104E90000E94A0278E910E94A0278E910E94A02799
:104EA0008E910E94A02785E90E94A0278F9180E023
:104EB00090E0A881B9818D939C938FEF0E94D12CB3
:104EC0000E94D32C0E94D22CAA81BB818C93A881F2
:104ED000B9810E948C2BAA81BB810C910F3F81E08C
:104EE00009F480E08F93A881B9810D911C91003065
:104EF00050E0150781E009F080E09F91892B88231D
:104F000011F40C945D27A881B9810D911C9100309A
:104F100050E0150711F00C949827ECE4FDE50E9491
:104F2000252C0E94312C7091CF0070647093CF00BB
:104F3000AA81BB818C91AA85BB858C930C94A527F3
:104F40008FB9779BFECF8FB1089587E0481A8827E5
:104F5000580A269608955A924A9284E298E0A42D1F
:104F6000B52D8D939C9382E00E94792B5A924A92A0
:104F700080E0A42DB52D8C9381E00E94792B0E94B6
:104F8000242A249683E00E94752BEF93FF93ECE88C
:104F9000F1E00E94B22CFF91EF91BB27A0E38C912E
:104FA00082FBDEF789E190E00E94DE2C5A924A9261
:104FB00080E298E0A42DB52D8D939C9382E00E9411
:104FC000792B5A924A9280E0A42DB52D8C9381E0E2
:104FD0000E94792B0E94242A249683E00E94752B3C
:104FE00089E190E00E94DE2C0E94AC28089582E0C6
:104FF0000E94ED2C00E011E0AA81BB814D91552764
:105000000E94F82BA881B9810D931C93A881B981C6
:105010000D911C91AA81BB814D915527040F151F3D
:10502000A881B9810D931C935A924A92AA81BB819F
:105030008D919C91A42DB52D8D939C9382E00E941F
:10504000792B5A924A928BE0A42DB52D8C9381E056
:105050000E94792B0E94242A249683E00E94752BBB
:105060005A924A9280E298E0A42DB52D8D939C939C
:1050700082E00E94792B5A924A9280E0A42DB52DAD
:105080008C9381E00E94792B0E94242A249683E04D
:105090000E94752B82E0481A8827580A22960895A4
:1050A00082E00E94ED2C00E110E0AC81BD814D91C9
:1050B00055270E94F82BA881B9810D931C93A881D4
:1050C000B9810D911C91AA81BB814D915527040F87
:1050D000151FA881B9810D931C935A924A92AA81F7
:1050E000BB818D919C91A42DB52D8D939C9382E0D5
:1050F0000E94792B5A924A9282E0A42DB52D8C936E
:1051000081E00E94792B0E94242A249683E00E9449
:10511000752B82E0481A8827580A229608955A92D9
:105120004A92AA81BB818D919C91A42DB52D8D931E
:105130009C9382E00E94792B5A924A9283E0A42D9C
:10514000B52D8C9381E00E94792B0E94242A24960D
:1051500083E00E94752B089581E00E94ED2C81E090
:105160000E94ED2CC49AD898C29880E0A881B98199
:105170008C9380E0AA81BB818C93AA81BB810C9126
:105180000F3118F011F00C94E12891E0A881B98159
:105190000E94C02C91E0A881B9810E94C02C91E0AE
:1051A000A881B9810E94C02C91E0A881B9810E9498
:1051B000C02CAA81BB818C918F5F8C9311F00C94D1
:1051C000BD28C29AD89A82E0481A8827580A24969D
:1051D000089581E00E94ED2C5A924A9280E298E074
:1051E000A42DB52D8D939C9382E00E94792B5A9229
:1051F0004A9280E0A42DB52D8C9381E00E94792BFA
:105200000E94242A249683E00E94752BAA81BB81E8
:105210000C91003011F00C941C295A924A9280E0B3
:10522000A42DB52D8C9381E00E94792B0E949629A4
:10523000229681E00E94752BAA81BB810C910130DE
:1052400011F00C9432295A924A9285E6A42DB52D7C
:105250008C9381E00E94792B0E949629229681E00E
:105260000E94752BAA81BB810C91023011F00C9425
:105270005F295A924A9283E6A42DB52D8C9381E042
:105280000E94792B0E949629229681E00E94752B1C
:1052900088EC90E00E94DE2C5A924A9280E0A42D85
:1052A000B52D8C9381E00E94792B0E94962922963D
:1052B00081E00E94752B82E390E00E94DE2CAA819F
:1052C000BB810C91033011F00C9488295A924A92B8
:1052D00082E6A42DB52D8C9381E00E94792B0E944B
:1052E0009629229681E00E94752B80E991E00E9428
:1052F000DE2C5A924A9280E0A42DB52D8C9381E049
:105300000E94792B0E949629229681E00E94752B9B
:105310008AE090E00E94DE2C8AE090E00E94DE2C81
:1053200081E0481A8827580A2296089581E00E9451
:10533000ED2CC49AD898C298AA81BB810C910030F8
:1053400018F011F00C94A6290C94E02983E5A881AB
:10535000B9818C9391E0A881B9810E94C02C8FEE15
:10536000A881B9818C9391E0A881B9810E94C02C59
:105370008EE6A881B9818C9391E0A881B9810E94C1
:10538000C02C91E0AA81BB810E94C02C80E0A88142
:10539000B9818C9391E0A881B9810E94C02C91E0E1
:1053A000A881B9810E94C02C91E0A881B9810E9496
:1053B000C02C91E0A881B9810E94C02C0C941C2AB9
:1053C00085E4A881B9818C9391E0A881B9810E947C
:1053D000C02C88E7A881B9818C9391E0A881B9811C
:1053E0000E94C02C89E6A881B9818C9391E0A881A4
:1053F000B9810E94C02C84E7A881B9818C9391E087
:10540000A881B9810E94C02C80E0A881B9818C93C9
:1054100091E0A881B9810E94C02C91E0A881B98156
:105420000E94C02C91E0A881B9810E94C02C91E01B
:10543000A881B9810E94C02CC29AD89A81E0481AEA
:105440008827580A2296089581E00E94ED2CC29A7E
:10545000D8985A924A9282E0A42DB52D8C9381E07F
:105460000E94792B0E94D92A229681E00E94752BF6
:105470005A924A92AC81BD818C91A42DB52D8C930A
:1054800081E00E94792B0E94D92A229681E00E9415
:10549000752BAC81BD8111968C91A881B9818C93BB
:1054A0005A924A92AA81BB818C91A42DB52D8C93DE
:1054B00081E00E94792B0E94D92A229681E00E94E5
:1054C000752BAC81BD818C91A881B9818C935A9246
:1054D0004A92AA81BB818C91A42DB52D8C9381E039
:1054E0000E94792B0E94D92A229681E00E94752B76
:1054F000D89A81E0481A8827580A2296089581E0B0
:105500000E94ED2C81E00E94ED2C82E00E94ED2CA7
:10551000C29AD8985A924A9283E0A42DB52D8C93C2
:1055200081E00E94792B0E94D92A229681E00E9474
:10553000752B5A924A92A885B9858C91A42DB52DC8
:105540008C9381E00E94792B0E94D92A229681E0D7
:105550000E94752BEC81FD81FA93EA930E94DF2A69
:105560002296EA81FB81FA93EA930E94DF2A22962F
:10557000D89AAC81BD810D91112740E051E00E9485
:10558000F82BA881B9810D931C93A881B9810D9145
:105590001C91AA81BB814D915527040F151FA88529
:1055A000B9850D931C9384E0481A8827580A2696DB
:1055B000089591E0A881B9810E94C02C089581E0EE
:1055C0000E94ED2C91E0A881B9810E94B52CA881A0
:1055D000B9818C91AA81BB818C9381E0481A88277C
:1055E000580A2296089582E00E94ED2C81E00E94E4
:1055F000ED2CC49ABB27A0E38C9182FBDEF7C29806
:10560000AC81BD810D911C91003052E0150711F065
:105610000C94422B81E090E0AA81BB818D939C93F6
:1056200080E0A881B9818C93A881B9810C910F3059
:1056300018F011F00C94402BBB27A0E38C9182FB57
:10564000DEF790E2AA81BB81AD90BC90A9EDB0E0FD
:10565000AA0DBB1D0E94C02CAA81BB810D911C917B
:1056600040E250E0040F151FAA81BB810D931C93EB
:10567000A881B9818C918F5F8C9311F00C94142BBD
:105680000C946E2B81E090E0AA81BB818D939C935A
:10569000AC81BD814D915C91AA81BB810D911C9122
:1056A0000417150718F011F00C946E2BBB27A0E31C
:1056B0008C9182FBDEF7C29A91E0AA81BB81AD900A
:1056C000BC90A9EDB0E0AA0DBB1D0E94C02CAA8120
:1056D000BB810E948C2B11F00C94482BC29A83E062
:1056E000481A8827580A24960895481A8827580A7D
:1056F0000895480E8827581E08950D911D912D91EB
:105700003C9181E0080F8827181F281F381F3C9301
:105710002E931E930E930895ED91FC913196FC9378
:10572000EE930895ED91FC913197FC93EE930895DB
:105730000D911D912D913C91015010402040304021
:105740003C932E931E930E9308954091DB0250914B
:10575000DC020DE815E30E94B92B49E156E3040F82
:10576000151F0093DB021093DC02498158810C94D1
:10577000DE2B08D03DD000FC10D0089503D01ED001
:1057800001F8F9CF0024E89457FF02C009D06894CB
:1057900000F80BD010F80124089502D009D0089524
:1057A000509540954F5F5F4F0895E89417FF089517
:1057B000009510950F5F1F4F68940895352F242F83
:1057C000E894452B11F468940895512F402F002739
:1057D000112780E1440F551F001F111F021B130BDF
:1057E000416018F4020F131F4E7F8A9599F70895B0
:1057F0000F92049F202C312C419F300C509F030CA2
:10580000022D102D0F900895C8950D92319600200D
:10581000D9F708958F938D918823E9F711978F9188
:10582000089581E05F9B8827089588275F9B0895EE
:1058300000C05F9BFECF8CB10895A8E6B7E08D91C4
:10584000882311F011D0FBCF08950E94F32C802DF6
:1058500011F00AD0FACF08958D9106D03A95E1F76C
:1058600008958DE001D08AE05D9BFECF8CB908954C
:1058700088EE93E0A3D03197D9F7089550D00AD09D
:1058800000FC05D008954BD020D001F8F9CF52D0BC
:105890005AD00895842F952FA62FB72F4427552728
:1058A00066277727F1E2889409C020F4480F591F32
:1058B0006A1F7B1F7695679557954795379527956E
:1058C00017950795FA9589F70895842F952FA62F98
:1058D000B72FE894452B462B472B11F46894089575
:1058E000402F512F622F732F002711272227332794
:1058F000F0E2440F551F661F771F001F111F221F64
:10590000331F081B190B2A0B3B0B416028F4080FAF
:10591000191F2A1F3B1F4E7FFA9559F7089500243F
:10592000E89477FF02C006D0689400F809D010F818
:105930000124089512D04F5F5F4F6F4F7F4F08953E
:10594000E89437FF089500951095209530950F5FE6
:105950001F4F2F4F3F4F6894089540955095609585
:10596000709508953197F1F708950E94D12C8C918C
:105970000E94D32C8D939A95D1F70E94D22C089532
:105980000E94D12C8D910E94D32C9A95D9F70E9418
:10599000D22C0895BF9ABE98C69ABD9A80E58DB95B
:1059A0000895089508958FB9779BFECF8FB108951C
:1059B000689462F80895E89462F80895EF93FF936D
:1059C000EE27E82BE92B31F0E0EDF7E03197F1F726
:1059D0000197D1F7FF91EF9108955A924A92480E9C
:1059E0008827581E0895C895319600200895819102
:1059F00004D08D938823D9F70895813618F08B371A
:105A000008F48F7D089580E30EF4839508952E2E7B
:105A10003F2E992781918D3209F093958823D1F7F4
:105A20009A95E22DF32D112361F0091718F011F06A
:105A3000101B01C0191B28F021F080E28D931A95EC
:105A4000E9F780818D3219F48D93319604C02223B9
:105A500011F08BE28D93091738F031F0091B21F01A
:105A600080E38D930A95E9F781918D938823E1F77F
:105A7000332351F0EA2FFB2F319633958E91829389
:105A80003A95E1F78EE28C930895040F151F261FB7
:105A9000371F0895041B150B260B370B08950417A9
:105AA0001507260737070895000F111F221F331F00
:105AB000089500951095209530950F5F1F4F2F4F3B
:105AC0003F4F0895019110810EC0019111912191D4
:105AD00030810BC00191108117FF05C03FEF2FEF00
:105AE00004C0008111272227332737FF03C0E1DFDD
:105AF0008DE28D93CF93DF93CF92DF92EF92AA2422
:105B0000BB24CC24DD24EE2440E2CAE0DD2755E0AE
:105B100093E38881890F87FD9F7083FD907F891BA8
:105B200089935A95A9F7C0DFAA1CBB1CCC1CDD1CAD
:105B3000EE1C4A9551F7E894EFE0FF2782910ED0D2
:105B4000EB30E0F71EF068948A2D0CD088278D93F7
:105B5000EF90DF90CF90DF91CF910895982F8295AD
:105B600001D0892F8F70805D26F0803309F408956D
:105B700068948D93089588278D93089581918D93CE
:105B80008823E1F7089509919191992351F08A951D
:105B9000D9F7319781918D930A9519F08823D1F720
:105BA0000895E9CFE199FECFEEBBFFBB3196089592
:105BB00091E001C092E07B3751F47FB7F894F2DFB7
:105BC0008D918DBBE29AE19A9A95C9F77FBF7727AD
:105BD000089591E001C092E0E5DFE09A8DB38D93E6
:105BE0009A95D1F70895FF93881BF9E0001FFA9565
:105BF00011F4FF910895881F841B18F4840F889472
:105C0000F5CF0894F3CF689401C0E894AF93BF93A5
:105C10008D9116F0919103C00E94F32C902D89175D
:105C200018F011F48823A1F7BF91AF9108954D505A
:105C3000335354414D50205265616C6974792D5332
:105C40007973203438352E3000005300500045451C
:105C500070726F6D20002C004D4D4320696E697489
:105C600020007265747279202E2E2E00445350202D
:105C7000696E697420004F005A00590057005200A5
:105C8000480021004E0042005800440045005600E4
:105C90004D00540049004C00434F4E464947000018
:105CA0002000442000002E006F6B00004E6F206328
:105CB000617264004261642063617264000050613B
:105CC00072746974696F6E2074797065203A00008F
:105CD000506172746974696F6E2073746172743A82
:105CE0000000536563742F636C75737465722020B4
:105CF0003A00526F6F74203A00005265616420656B
:105D000072726F7220310000526561642065727298
:105D10006F722032206F6E20736563746F723A2049
:105D2000000052656164206572726F72203300005A
:105D300052656164206572726F7220340000526592
:105D40006164206572726F72203500005265616473
:0A5D50002074696D656F7574000022
:00000001FF
